:100000000C94D5060C94F4060C94F4060C94F406A7
:100010000C94F4060C94F4060C94F4060C94F40678
:100020000C94F4060C94F4060C94A32C0C94792DE7
:100030000C94B9260C94F4060C94F4060C94F40673
:100040000C94F4060C94F4060C94F4060C94F40648
:100050000C94F4060C9441270C94F4060C94F406CA
:100060000C94F4060C946A200C94F4060C94F40698
:100070000C94F4060C94F4060C94F4060C94F40618
:100080000C94F4060C94F4060C94F4060C94F40608
:100090000C94F4060C94F406000B000B2C0B2C0BA8
:1000A000940BB20BD80CD80CCB0B640C750C750CE4
:1000B000E422D222EB225D2298239823CF22982398
:1000C0009823182398232C23782398239823982364
:1000D00098234C2398239823492398230423982377
:1000E0009823922392239223922392239223922362
:1000F0009223922394239823E422C72298239823BF
:100100009823982398239823982398239823982317
:10011000942398239823CF229823902390239023ED
:100120009023902390239023902390239423EA2DCF
:10013000112E092F112E092F5D2E802E092FD72E5B
:10014000E62E290000003A003B003C003D00000084
:100150003E003F0040004100420043004400450093
:100160004600470048000000A800AC00AB00AE000D
:10017000000000000000000000000000000000007F
:10018000000000000000000000000000000000006F
:10019000000000000000000000000000000035002A
:1001A0001E001F0020002100220023002400250043
:1001B000260027002D002E0000002A0049004A00DA
:1001C0004B00000053005400550056002B00000067
:1001D00014001A000800150017001C0018000C007D
:1001E000120013002F00300031004C004D004E0073
:1001F00000005F00600061000000390000000400A2
:100200001600070009000A000B000D000E000F0089
:10021000330034002800000000000000000000004F
:100220005C005D005E0057000000E1001D001B0047
:1002300006001900050011001000360037003800D4
:100240000000E10000000000520000000000590022
:100250005A005B000000E000E3000000E200000044
:1002600000002C00000000000000E200E30000009D
:100270006500E000500051004F00000062000000E7
:100280006300580000000000000000000000F100C2
:10029000F300F20000000000000000000000000079
:1002A000000000000000000000000000000000004E
:1002B000000044454255473A2064697361626C65A9
:1002C000642E0A0044454255473A20656E61626CCF
:1002D00065642E0A000A0025303258006C65645FA0
:1002E0007461736B3A20004F6E6573686F743A20C7
:1002F0006163746976653A2025640A000A00253036
:1003000033326C62003A200025303258000A722FD6
:100310006320303132333435363738394142434443
:10032000454630313233343536373839414243442B
:1003300045460A00290A002575002F002575005D35
:10034000280025640020002564002000256400208A
:10035000002564007C0025303258006D6F75736590
:100360006B6579205B62746E7C78207920762068DA
:100370005D287265702F61636C293A205B002063F1
:100380006F6D6D616E643A2025582C20726573750F
:100390006C743A2025582C206572726F723A2025B1
:1003A00058200A00707332206D6F75736520656E7A
:1003B00061626C652064617461207265706F727433
:1003C000696E67007073325F6D6F7573653A206692
:1003D00061696C20746F20676574206D6F7573653B
:1003E000207061636B65740A0020726573756C74AC
:1003F0003A2025582C206572726F723A20255820B9
:100400000A007073325F6D6F7573655F696E697432
:100410003A20726561642044657649440020726523
:1004200073756C743A2025582C206572726F723A7D
:10043000202558200A007073325F6D6F7573655FF9
:10044000696E69743A2072656164204241540020EB
:10045000636F6D6D616E643A2025582C2072657350
:10046000756C743A2025582C206572726F723A2090
:100470002558200A007073325F6D6F7573655F6970
:100480006E69743A2073656E64696E672072657375
:10049000657400706275663A2066756C6C0A00506F
:1004A0005332205553415254206572726F723A2074
:1004B0002530325820646174613A20253032580A60
:1004C00000313A0964656C6179282A31306D7329ED
:1004D0003A2025750A323A09696E74657276616C44
:1004E000286D73293A2025750A333A096D61785FC2
:1004F00073706565643A2025750A343A0974696D2C
:10050000655F746F5F6D61783A2025750A353A0929
:10051000776865656C5F6D61785F73706565643A77
:100520002025750A363A09776865656C5F74696DD0
:10053000655F746F5F6D61783A2025750A00703AC7
:10054000097072696E742076616C7565730A643A1D
:10055000097365742064656661756C74730A7570DF
:100560003A092B310A646E3A092D310A6C743A0942
:100570002B31300A72743A092D31300A4553432F1A
:10058000713A09717569740A0A7370656564203D72
:100590002064656C7461202A206D61785F737065DA
:1005A0006564202A2028726570656174202F20748C
:1005B000696D655F746F5F6D6178290A7768657230
:1005C000652064656C74613A20637572736F723D67
:1005D00025642C20776865656C3D25640A53656544
:1005E00020687474703A2F2F656E2E77696B69706E
:1005F000656469612E6F72672F77696B692F4D6F24
:100600007573655F6B6579730A004D3E20004D255B
:10061000753A25733E20003F0A003D2025750A00EB
:100620003F0A0064656661756C74730A0025750A7B
:10063000003F0A000A092D2056616C756573202D54
:100640000A00710A000A092D204D6F7573656B65EC
:1006500079202D0A003F00433E20004C25640A000B
:100660000A092D20537461747573202D0A686F7305
:10067000745F6B6579626F6172645F6C6564732827
:10068000293A20253032580A6B6579626F617264AD
:100690005F70726F746F636F6C3A20253032580A46
:1006A0006B6579626F6172645F69646C653A20257D
:1006B0003032580A6B65796D61705F636F6E666981
:1006C000672E6E6B726F3A20253032580A74696D4E
:1006D00065725F72656164333228293A20253038AB
:1006E0006C580A000A092D2056657273696F6E20D6
:1006F0002D0A5649443A2030783132333428514D4E
:100700004B29205049443A20307835363738283143
:1007100030384B65792D547261636B706F696E74FC
:1007200029205645523A203078303030310A42552F
:10073000494C443A20202846656220323720323026
:100740003232290A4F5054494F4E533A204C5546A5
:1007500041204D4F5553454B455920455854524122
:100760004B455920434F4E534F4C4520434F4D4D21
:10077000414E44204E4B524F20313032340A4743D1
:10078000433A20352E342E30204156522D4C4942CA
:10079000433A20322E302E30204156525F41524390
:1007A000483A2061767235310A000A092D20436FDC
:1007B0006E736F6C65202D0A4553432F713A097192
:1007C0007569740A6D3A096D6F7573656B65790AA1
:1007D000000A092D204D61676963202D0A443A09FA
:1007E0004465627567204D65737361676520546F5A
:1007F00067676C650A583A094D61747269782044DC
:1008000065627567204D6F646520546F67676C651E
:10081000202D2053686F77206B6579707265737334
:10082000657320696E206D617472697820677269E2
:10083000640A4B3A094B6579626F617264204465C2
:1008400062756720546F67676C65202D2053686F51
:1008500077206B65797072657373207265706F7243
:10086000740A4D3A094465627567204D6F7573656A
:1008700020546F67676C650A563A0956657273694A
:100880006F6E0A533A095374617475730A433A09D7
:10089000416374697661746520436F6E736F6C6534
:1008A000204D6F64650A46312D4631303A09537741
:1008B0006974636820746F204C6179657220302DF3
:1008C000392028463130203D204C30290A302D393E
:1008D0003A0953776974636820746F204C617965B5
:1008E0007220302D390A47524156453A09537769EB
:1008F00074636820746F204C617965722030202801
:10090000616C7465726E617465290A423A094A75B0
:100910006D7020746F20426F6F746C6F61646572CC
:100920000A4553433A094A756D7020746F20426F2F
:100930006F746C6F616465722028616C7465726E8F
:10094000617465290A453A095072696E74204545FB
:1009500050524F4D2053657474696E67730A425349
:10096000504143453A09436C6561722045455052F8
:100970004F4D0A4E3A094E4B524F20546F67676CE9
:10098000650A006B65796D61705F636F6E6669679C
:100990002E7261773A20253032580A2E73776170B3
:1009A0005F636F6E74726F6C5F636170736C6F63A3
:1009B0006B3A2025750A2E636170736C6F636B5FF1
:1009C000746F5F636F6E74726F6C3A2025750A2EB8
:1009D000737761705F6C63746C5F6C6775693A20E4
:1009E00025750A2E737761705F7263746C5F72672E
:1009F00075693A2025750A2E737761705F6C616C9A
:100A0000745F6C6775693A2025750A2E737761707B
:100A10005F72616C745F726775693A2025750A2E82
:100A20006E6F5F6775693A2025750A2E737761705E
:100A30005F67726176655F6573633A2025750A2E7C
:100A4000737761705F6261636B736C6173685F621F
:100A500061636B73706163653A2025750A2E6E6B56
:100A6000726F3A2025750A0064656275675F636F6F
:100A70006E6669672E7261773A20253032580A2EE9
:100A8000656E61626C653A2025750A2E6D6174721F
:100A900069783A2025750A2E6B6579626F617264F8
:100AA0003A2025750A2E6D6F7573653A2025750AF3
:100AB000006565636F6E6669673A0A6465666175AD
:100AC0006C745F6C617965723A2025750A003F008D
:100AD0004E4B524F3A206F66660A004E4B524F3AC9
:100AE000206F6E0A000A6D6F7573653A206F666637
:100AF0000A000A6D6F7573653A206F6E0A000A6B03
:100B00006579626F6172643A206F66660A000A6BEB
:100B10006579626F6172643A206F6E0A000A6D61D6
:100B2000747269783A206F66660A000A6D617472A1
:100B300069783A206F6E0A000A64656275673A2028
:100B40006F66660A000A64656275673A206F6E0A0E
:100B5000000A0A4A756D70696E6720746F20626FB3
:100B60006F746C6F616465722E2E2E2000433E20E0
:100B700000436C656172696E6720454550524F4D68
:100B80000A000A002530325820006B6579626F61D7
:100B900072645F7265706F72743A200064656C5F96
:100BA0006B65795F6269743A2063616E27742064B3
:100BB000656C3A20253032580A006164645F6B65C9
:100BC000795F6269743A2063616E2774206164649E
:100BD0003A20253032580A005B735D005B575D0098
:100BE0005B535D005B525D005B445D005B435D00F9
:100BF00024033100300038004B00650079002D00DF
:100C000054007200610063006B0070006F006900A7
:100C10006E0074000000080351004D004B000000FE
:100C20000403090409025B00030100A0FA0904009F
:100C30000001030101000921110100012240000708
:100C400005810308000109040100010300000009F7
:100C5000211101000122B6000705820320000109CD
:100C600004020002030000000921110100012222F8
:100C7000000705830320000107050303200001127C
:100C80000100020000000834127856010001020041
:100C9000010631FF0974A1010975150026FF0095B1
:100CA00020750881020976150026FF009520750839
:100CB0009102C005010902A10185020901A10005F7
:100CC00009190129081500250195087501810205FA
:100CD00001093009311581257F95027508810609C2
:100CE000381581257F950175088106050C0A3802A3
:100CF0001581257F950175088106C0C00501098011
:100D0000A101850319012AB700150126B700950135
:100D100075108100C0050C0901A101850419012A83
:100D2000A002150126A002950175108100C00501E1
:100D30000906A1018506050719E029E71500250127
:100D40009508750181020507190029EF1500250195
:100D500095F07501810205081901290595057501B0
:100D60009102950175039101C005010906A10105D4
:100D70000719E029E71500250195087501810295FD
:100D800001750881010507190029FF150026FF00DC
:100D90009506750881000508190129059505750155
:100DA0009102950175039101C00011241FBECFEF80
:100DB000D0E2DEBFCDBF12E0A0E0B1E0E4E9FFE5A4
:100DC00000E00BBF02C007900D92A630B107D9F723
:100DD00023E0A6E0B2E001C01D92A63FB207E1F712
:100DE0000E946C190C94C82F0C940000FF93EF9391
:100DF000E0910602F0910702309709F00995EF9112
:100E0000FF910895FC018591803011F0EFDFFBCF59
:100E10000895FF27E0E230E247FF0CC0419597FFBD
:100E200009C0EDE26095709580959095611D711DEA
:100E3000811D911D27FF02C0219530E350E2AA27B2
:100E4000660F771F881F991FAA1FA41710F0A41BF5
:100E500063955A95A9F7AA3008F0A95FA05DAF93F2
:100E6000F395611571058105910541F7ED3211F496
:100E7000EF93F395F21718F43F93F395FBCF8F910F
:100E8000B5DFFA95E1F70895E991F9918591803000
:100E900021F0853219F0AADFF9CF089520E0E89417
:100EA00055915532C1F3503311F4689455915A332A
:100EB00048F4505390F3220F022E220F220F200DE0
:100EC000250FF4CF0EF4219589919991533619F39A
:100ED000533729F1533559F1BC0188279927E894F4
:100EE0005C3621F48991999168945591543639F47E
:100EF00046EF7EF077FF0DC08FEF9FEF0AC05537AA
:100F00004AE039F0583540E121F0523642E009F02C
:100F10000895FF93EF937DDFEF91FF91B7CFFF939C
:100F2000EF93FC0181918030B9F360DFFBCFFF9339
:100F3000EF9368DFF1CFDF93CF93CDB7DEB7259680
:100F4000A3DFCF91DF91089581E0089581E00895B6
:100F50000C94A60708950C94AA071F93CF93DF93D0
:100F600000D000D01F92CDB7DEB749835A836B8380
:100F70003091090289819A81311114C0662359F098
:100F8000222349F00E94150F182F682F89819A811A
:100F90000E94BE0E03C00E94E90E182F69817A815B
:100FA000812F04C00E94150F69817A810F900F90E4
:100FB0000F900F900F90DF91CF911F910C94851699
:100FC000FC01262F408151816281738184810C94C0
:100FD000AD0781E00895CF93DF93EC0160E00E94BC
:100FE000E007BE01DF91CF910C94AB070C94FF1783
:100FF0000C94FB1708950E94680D0E94FA072FEFCA
:1010000084E39CE0215080409040E1F700C0000064
:101010000C9467270F931F93CF93DF938C0161E0AC
:101020000E94E007EC01B8010E94A807882309F498
:101030005BC0B801CE010E94A524882309F454C0E6
:10104000B801CE010E94841C882309F44DC0B80168
:10105000CE010E940124882309F446C0F801828150
:101060008823D9F1CF3D8CE5D80779F140F4C1153B
:10107000FCE5DF0791F0C130DC4591F02EC0CC35A6
:10108000EDE5DE0741F1CD35FDE5DF0709F1CB35B3
:10109000DD4519F50E94AC1320C00E94FB0724C057
:1010A00080912903C82FC095C170C0FB80F980933F
:1010B0002903CC2329F084EC92E00E94020714C09B
:1010C00082EB92E00E94020710C00E945A140CC0EA
:1010D0000E94A31302C00E94AF13C801DF91CF91F9
:1010E0001F910F910C94A407C0E08C2FDF91CF913A
:1010F0001F910F9108950E9499260C94E4080E9474
:10110000E7080C949F268295982F937344E0949F50
:10111000900111248C7C86958695282B822F8575CD
:10112000880F2A7A2695822B0895CF93DF93D92FA3
:101130000E948308C82F8D2F0E9483082C2F30E037
:10114000322F2227A901482BCA01DF91CF910895A0
:10115000CF92DF92EF92FF920F931F93CF93DF9383
:101160006B017C01CB010E949508EC01C7010E9434
:101170009508AC01CE01A0E0B0E0DC0199278827FA
:1011800060E070E08C019D01042B152B262B372B82
:10119000C901B801DF91CF911F910F91FF90EF909E
:1011A000DF90CF90089508950C94D30881E00895BE
:1011B0000C94D6080895CF93C82F0E94D4088C2F82
:1011C0000E94D808CF91089580E00C94DB080E941B
:1011D00001250C94DB08CF930E940125C82F809134
:1011E0000802C81741F1C09308028091290382FFC9
:1011F0001EC080FF04C08CED92E00E940207809127
:10120000290380FF0CC01F92CF9387ED92E09F933C
:101210008F930E949B070F900F900F900F908091DB
:10122000290380FF04C085ED92E00E9402078C2F05
:10123000CF910C94DB08CF910895CF93DF93CDB776
:10124000DEB72B970FB6F894DEBF0FBECDBF4F832E
:10125000588769877A878B8761110E94DB129E010C
:101260002F5F3F4F86E0F90111928A95E9F785E0FB
:10127000FE013796D90101900D928A95E1F7898197
:101280009A814C815D81452B31F09F3F31F491E093
:101290008F3F19F403C091E001C090E090FF09C0B6
:1012A00049815A816B817C818D819E810E94FC11D4
:1012B00005C0C9010E94E9078111F2CF2B960FB634
:1012C000F894DEBF0FBECDBFDF91CF910895FC0132
:1012D000808191810E94570F089570E02091A103B1
:1012E0003091A203882319F0622B732B04C0609500
:1012F0007095622373237093A2036093A1030895F2
:10130000CF93882309F4A9C0C82F8238C1F40E9462
:10131000012581FDA2C069E3809102019091030142
:101320000E9454260E94FD122FEF81EE94E021507E
:1013300080409040E1F700C0000069E319C08338A5
:1013400001F50E94012580FD88C063E580910201BE
:10135000909103010E9454260E94FD122FEF81EE0E
:1013600094E0215080409040E1F700C0000063E528
:1013700080910201909103010E945F26CF910C940D
:10138000FD128438C1F40E94012582FD66C067E425
:1013900080910201909103010E9454260E94FD1247
:1013A0002FEF81EE94E0215080409040E1F700C0A3
:1013B000000067E4DDCF8CEF8C0F813AF8F48C2FBE
:1013C0000E94AA23811149C06C2F80910201909143
:1013D00003010E94B225882349F06C2F80910201FD
:1013E000909103010E945F260E94FD126C2F809154
:1013F0000201909103010E945426C0CF80E28C0F1D
:10140000883048F4C77081E001C0880FCA95EAF7B8
:101410000E94BE12B3CFEBE5EC0FE33040F4F0E0F6
:10142000E95BFE4F808190E0CF910C947025E8E558
:10143000EC0FE73150F4F0E0EE0FFF1FE75EFE4FD8
:1014400080819181CF910C948625CD3E30F08C2FF8
:101450000E94F119CF910C94C31ACF91089588235B
:1014600009F464C0823879F40E94012581FF5EC0CE
:1014700069E380910201909103010E9454260E9429
:10148000FD1269E310C08338B1F40E94012580FF8A
:101490004DC063E580910201909103010E945426A2
:1014A0000E94FD1263E580910201909103010E9468
:1014B0005F260C94FD12843879F40E94012582FF86
:1014C00035C067E480910201909103010E94542687
:1014D0000E94FD1267E4E7CF9CEF980F913A10F459
:1014E000682FE1CF90E2980F983050F4877091E028
:1014F00001C0990F8A95EAF7892F0E94C412D9CFAB
:101500009BE5980F933020F480E090E00C947025D8
:1015100098E5980F973120F480E090E00C948625B0
:101520008D3E20F00E944C1A0C94C31A08951F930C
:10153000CF93DF93182FEB010E948009209741F091
:101540008FE99FE00197F1F700C000002197F6CFE7
:10155000812FDF91CF911F910C942F0A893319F0BD
:1015600060E070E002C060E570E00C94970A8823A8
:1015700021F00E94BE120C94FD120895882321F0E0
:101580000E94C4120C94FD120895CF92DF92EF9244
:10159000FF920F931F93CF93DF937C01D62FC72F1A
:1015A000FC011281058102950F700E94B4128823FC
:1015B000B9F01123A9F08C2F807F803421F080E2D4
:1015C0008D0F883068F08091A40382FD09C082E00D
:1015D0000E945D130E94B41291E0D82ED92601C05A
:1015E000D12CCC2EC2948FE0C8228C2D90E08C3070
:1015F000910508F0DDC1FC01E45BFF4F0C945C2F0A
:101600008C2F807FCF70882311F0C295C07F11236B
:1016100099F0CC2309F4B8C180E28D0F883010F026
:10162000D11104C08C2F0E94BE1203C08C2F0E94C7
:10163000CE120E94FD12A8C18D2F0E942F0ACC232A
:1016400009F4B6C180E28D0F883038F1DD2329F12D
:101650008C2F0E94D41224C08C2F807FCF708032B8
:1016600011F0C295C07FDD2319F0D130A1F13DC04A
:101670008091A40382FF17C0112349F0CC2329F0E5
:101680008C2F0E94BE120E94FD1280E07EC180E07D
:101690000E942F0ACC2309F48BC18C2F0E94C41204
:1016A0000E94FD1285C1112371F0002341F0013029
:1016B00031F40E94DE128C2B0E94E61279C10E9446
:1016C000DE128C2B1DC0002319F0013009F470C10B
:1016D0000E94F31225C0112321F0063008F068C1E2
:1016E0000EC0053008F064C11BC0112361F0002357
:1016F00031F0F701858180FF47C18F7085838C2F82
:101700000E94B70A55C1002359F0D93309F04DC1E1
:10171000FFEF07EE13E0F15000401040E1F743C146
:101720008C2F0E94BE0A44C18C2F869586958370AB
:1017300019F0813061F03CC1112321F08D2F9C2FD5
:10174000937002C080E090E00E94702539C111239F
:1017500021F08D2F9C2F937002C080E090E00E94BA
:1017600086252EC18D2F112319F00E94F11902C078
:101770000E944C1A8FE08D0F833050F461E070E0CE
:1017800001C0660F8A95EAF7812F0E946D0918C182
:101790000E94C31A15C18C2F837009F047C0111124
:1017A0000BC12D2F229526952770220F220F6D2F0A
:1017B0006F70862F90E0A0E0B0E0022E04C0880F8A
:1017C000991FAA1FBB1F0A94D2F7D4FF10C04FE085
:1017D00050E060E070E004C0440F551F661F771FA3
:1017E0002A95D2F7409550956095709503C040E0DA
:1017F00050E0BA01C695C695C3708A019B01082BBB
:10180000192B2A2B3B2BC901B801C23049F058F4DF
:10181000C13019F00E94D40DCFC00E94C20DCCC0BF
:101820000E94E60DC9C00E94C00DC6C0112319F068
:101830008C2F817001C08695882309F4BDC02D2F9F
:10184000229526952770220F220F6D2F6F70862FFD
:1018500090E0A0E0B0E0022E04C0880F991FAA1FFC
:10186000BB1F0A94D2F7D4FF10C04FE050E060E0F5
:1018700070E004C0440F551F661F771F2A95D2F7EA
:10188000409550956095709503C040E050E0BA01D6
:10189000C695C695C3708A019B01082B192B2A2B6C
:1018A0003B2BC901B801C23049F058F4C13019F0DE
:1018B0000E94990E81C00E94870E7EC00E94AB0ECE
:1018C0007BC00E94FA0D78C0CF70112339F08C2FA5
:1018D0000E94200E8D2F0E94B70A6EC08D2F0E948D
:1018E000BE0A8C2F0E94410E67C0D23F21F128F41E
:1018F000D03F41F0D13FC1F043C0D33F19F1D43FB5
:1019000079F03EC0112341F0053008F051C08C2F12
:101910008F710E94660E4CC0063008F049C0F7CFA8
:101920008091A40382FF18C0112339F08C2F8F718E
:101930000E94200E3DC01123C9F38C2F8F710E948D
:10194000410E36C0112329F08C2F8F710E940B0E8F
:101950002FC00E94060E2CC0112349F0CF718C2F8E
:101960000E94200E63E08C2F0E94421321C081E070
:101970000E945D130230E0F082E00E945D1318C007
:10198000112331F0002391F28D2F0E94800910C0A5
:10199000002399F2D93349F41FEF27EE33E01150B9
:1019A00020403040E1F700C000008D2F0E942F0A38
:1019B00088EF8C0D843020F40E9401250E94DB0802
:1019C000DD20C9F00E94B01280FD15C0F70112821F
:1019D0000E94AA120E94200EC7010E941C0D0E94A4
:1019E000AA12DF91CF911F910F91FF90EF90DF909E
:1019F000CF900C94410EDF91CF911F910F91FF90EA
:101A0000EF90DF90CF9008950F931F93CF93DF93C4
:101A1000EC01688179818A810E94620F8C010E94A9
:101A2000BD0E0E94AE0DB801CE010E94C50ADF9125
:101A3000CF911F910F910895CF93DF93EC0198817F
:101A400089812B813C81232B31F08F3F31F481E060
:101A50009F3F19F403C081E001C080E080FD1DC0FC
:101A6000CE010E940A08811110C00E94B41288237E
:101A7000A1F08A81882389F08091A40382FD0DC0A2
:101A800082E0DF91CF910C945D13CE010E94040D92
:101A9000CE01DF91CF910C94EB07DF91CF910895A8
:101AA00080E090E00E94702580E090E00E94862512
:101AB0000E94DB120E94FD120E94761C0C94C31A35
:101AC00080910201909103010E946A260C94500DAE
:101AD0000E94CB120C94600D92959F70963079F015
:101AE00010F4925001C09A50923068F4803F69F02F
:101AF00018F4883E40F409C0843F29F406C0883EAB
:101B000020F0813F11F080E0089581E00895FC010C
:101B1000808191810E94570F0E946C0D0895CF9390
:101B2000DF9300D000D01F92CDB7DEB70F900F909B
:101B30000F900F900F90DF91CF910895CF93DF9387
:101B400000D000D000D0CDB7DEB726960FB6F894FF
:101B5000DEBF0FBECDBFDF91CF91089508950895E8
:101B60000C94AF0D0C94B00D0E94B20D60938102E5
:101B70007093820280938302909384020C94500DA0
:101B80000C94B40D0F931F93009181021091820267
:101B90002091830230918402602B712B822B932B36
:101BA0001F910F910C94B40D0F931F93009181021C
:101BB000109182022091830230918402602371236C
:101BC000822393231F910F910C94B40D0F931F93B5
:101BD000009181021091820220918302309184024F
:101BE00060277127822793271F910F910C94B40DC2
:101BF0000C94AF0D0E94F80D60937D0270937E02ED
:101C000080937F02909380020C94500D60E070E00E
:101C1000CB010C94FA0D0F931F9341E050E060E06C
:101C200070E08A019B0104C0000F111F221F331FA7
:101C30008A95D2F7C901B8011F910F910C94FA0D42
:101C40000F931F9341E050E060E070E004C0440F48
:101C5000551F661F771F8A95D2F780917D0290915C
:101C60007E02A0917F02B09180028A019B01082B25
:101C7000192B2A2B3B2BC901B8011F910F910C94F2
:101C8000FA0D0F931F9341E050E060E070E004C054
:101C9000440F551F661F771F8A95D2F740955095C0
:101CA0006095709580917D0290917E02A0917F0257
:101CB000B09180028A019B01082319232A233B2328
:101CC000C901B8011F910F910C94FA0D0F931F9346
:101CD00041E050E060E070E004C0440F551F661F13
:101CE000771F8A95D2F780917D0290917E02A09114
:101CF0007F02B09180028A019B01082719272A27B9
:101D00003B27C901B8011F910F910C94FA0D0F9355
:101D10001F9300917D0210917E0220917F023091ED
:101D20008002602B712B822B932B1F910F910C94AF
:101D3000FA0D0F931F9300917D0210917E02209166
:101D40007F023091800260237123822393231F91AD
:101D50000F910C94FA0D0F931F9300917D02109137
:101D60007E0220917F0230918002602771278227B6
:101D700093271F910F910C94FA0D089527E1929FDC
:101D8000800D1124E82FE695E695E695877051E0E1
:101D900001C0550F8A95EAF785E0E89FF00111240C
:101DA000E65FFD4F20E030E070E04081CB01022E85
:101DB00002C0969587950A94E2F7817081958427F1
:101DC0008523842781932F5F3F4F2530310569F7A5
:101DD000089527E1929F800D1124682F66956695DE
:101DE0006695982F977085E0689FB001112440E0B8
:101DF00050E080E0FB01E40FF51FE65FFD4F20811E
:101E000030E0092E02C0369527950A94E2F721703A
:101E10003327042E01C0220F0A94EAF7822B4F5F6A
:101E20005F4F4530510531F70895BF92CF92DF9251
:101E3000EF92FF920F931F93CF93DF938C01C0908B
:101E40007D02D0907E02E0907F02F090800280912F
:101E5000810290918202A0918302B0918402C82AEB
:101E6000D92AEA2AFB2ACFE1D0E0D701C6010C2EFD
:101E700004C0B695A795979587950A94D2F780FDEB
:101E800004C0219790F7B12C07C0BC2EB8018C2F4D
:101E90000E9498160197A9F38B2DDF91CF911F9186
:101EA0000F91FF90EF90DF90CF90BF900895CF9368
:101EB000DF93EC010E94150FBE010E949816DF917E
:101EC000CF9108951F93CF93DF93EB019091090277
:101ED000992321F0CB010E94570F13C0882349F0AA
:101EE000CB010E94150F182F682FCE010E94BE0E45
:101EF00004C0CB010E94E90E182FBE01812F0E9461
:101F00009816DF91CF911F9108951F93CF93DF9380
:101F1000C091850216E080918602C81799F0D0E042
:101F20001C9FF0011D9FF00D1124E957FD4F4081CA
:101F3000518162817381848195810E949E0D2196D9
:101F4000C770E9CFDF91CF911F9108954091B702FB
:101F50005091B8026091B9027091BA028091BB02AF
:101F60009091BC020C949E0DEF92FF920F931F93E1
:101F7000CF93DF938091BC0282958F7009F065C08A
:101F80008091B902882309F460C080918502F090A5
:101F900086021091B7020091B8026091BA02709166
:101FA000BB0291E01F3F09F090E0C0910001D09189
:101FB0000101292F96E0E92E8F1509F446C061151D
:101FC000710521F00F3F21F030E003C031E001C086
:101FD000322F90E030FD36C0E89EF001E99EF00D12
:101FE0001124DF01A957BD4F11963C911197301371
:101FF00029C03C91311326C012963C9112973111A1
:1020000021C013964D915C911497461B570B4C17AA
:102010005D07C0F48091BC028F7080618093BC0228
:10202000E457FD4F80818F708061808387EB92E061
:102030000E941C0DDF91CF911F910F91FF90EF90A7
:102040000C94850F01968770B7CFDF91CF911F91C8
:102050000F91FF90EF9008959F92AF92BF92CF9211
:10206000DF92EF92FF920F931F93CF93DF93CDB741
:10207000DEB761970FB6F894DEBF0FBECDBF8C01FF
:1020800085E0F801DE011D9601900D928A95E1F739
:10209000D8011296EC909091B702E091B80220918D
:1020A000BA023091BB022115310531F0EF3F31F416
:1020B00081E09F3F19F403C081E001C080E0B82FA8
:1020C000B1709B2E80FD47C1D8014C9111965C9157
:1020D00011971396AD90BC90149787EBC82E82E0B1
:1020E000D82EF090B902B501621B730B209100014C
:1020F00030910101FF2009F4D9C08091BC02621720
:10210000730708F095C0282F207F09F052C05E1396
:1021100013C0491311C0FE2CE1100EC08F708061F6
:102120008093BC020E94A60FC6010E941C0D8091E4
:10213000BC02F80185834DC1AB2831F05F3F31F41B
:1021400081E04F3F19F403C081E001C080E080FDD1
:1021500003C081E08E2502C080E090E0F82FF1708E
:10216000FF2E80FF1CC0809185022091860236E000
:10217000821709F40BC190E0389FF001399FF00DF0
:102180001124E957FD4F6181561306C06081461343
:1021900003C06281E61203C001968770E9CFFE2C6E
:1021A000EE2009F416C18091BC0281608093BC02CC
:1021B00054C05E1306C0491304C0E11002C0F80108
:1021C00099C0C8010E94870D882361F1EE2051F16A
:1021D0002091BC02822F82958F7090E0029774F05C
:1021E0008091B7029091B80298878F831986BB8639
:1021F000AA862C87CE0107960E941C0D86E0F80166
:10220000A7EBB2E001900D928A95E1F70E94B40F1E
:102210000E94A60F0AC05E1711F1C8010E94870D27
:1022200081112CC0C8010E941C0DFF24F394D1C061
:10223000282F207F81F77A2DB98AA88A6E2D898967
:102240000E948F0D87EB92E00E941C0D86E0D60164
:102250001D928A95E9F70E94A60FF12CBAC0491386
:10226000DCCFE110DACFF8018583C8010E941C0D94
:1022700086E0D6011D928A95E9F7ABC0EE2091F277
:102280002091BC02822F82958F7090E002970CF40F
:10229000B5CF8091B7029091B8029A8389831B824F
:1022A000BD82AC822E83CE010196A6CF6217730742
:1022B00008F044C0FE2CEE2009F4B4CF5E1330C009
:1022C00049132EC02091BC0220FD21C0822F82958F
:1022D0008F70482F50E041155105C9F0F801258352
:1022E0004F30510541F08F5F982F9295907F822F4C
:1022F0008F70892B8583C8010E941C0D86E0F80130
:10230000A7EBB2E001900D928A95E1F73CC086E020
:10231000F801A7EBB2E001900D928A95E1F759C060
:10232000C8010E94870D811169CF8091BC02816034
:102330008093BC02C8010E941C0D4BC07A2DB98A43
:10234000A88A6E2D89890E948F0D86E0D6011D9284
:102350008A95E9F718C0EE2009F464CFC8010E94FD
:10236000870DF82E882309F45DCF86E0F801A7EBEE
:10237000B2E001900D928A95E1F787EB92E00E941E
:1023800067090E94B40F0E94A60F23C04D875E8785
:102390008D859E850E94570F292F22952F70223000
:1023A00028F49F7039F0811105C00BC0243028F447
:1023B0009F7049F4805E883020F0C8010E941C0D97
:1023C0009F2CF92C06C0D80115969C91907F91F70F
:1023D000F8CF8F2D61960FB6F894DEBF0FBECDBF3C
:1023E000DF91CF911F910F91FF90EF90DF90CF90F1
:1023F000BF90AF909F9008951F93CF93DF93CDB779
:10240000DEB72C970FB6F894DEBF0FBECDBF4F835B
:10241000588769877A878B879C87CE0107960E94A9
:102420002C108823D1F09F8188852A853B85232B1A
:1024300031F08F3F31F481E09F3F19F403C081E018
:1024400001C080E080FD47C04F81588569857A854D
:102450008B859C850E949E0D3EC086E0FE013796CE
:10246000DE01119601900D928A95E1F7FF81E885D2
:102470006A857B856115710531F0EF3F31F481E0AC
:10248000FF3F19F403C081E001C080E080FD23C05C
:102490002091860230E0C90101968770992740910A
:1024A000850250E084179507F1F1F983EA837D8373
:1024B0006C8396E0929FD001939FB00D1124A95791
:1024C000BD4FFE01319601900D929A95E1F78093F0
:1024D00086020E94850F16E0809185029091860207
:1024E000891771F1189FC001112489579D4F0E94CF
:1024F0002C10882329F1E09185021E9FF001112400
:10250000E957FD4F408151816281738184819581BA
:102510000E949E0D8091850290E001968770992718
:1025200080938502D9CF0E94680D10928602109286
:102530008502E7EBF2E086E0DF011D928A95E9F77C
:102540002C960FB6F894DEBF0FBECDBFDF91CF91B2
:102550001F9108958091DD02859585958595089553
:102560008091DD02877008959091DD02977081E07F
:1025700009F480E00895809100030895909100038C
:10258000892B8093000308958095909100038923FF
:102590008093000308951092000308959091FF0224
:1025A000892B8093FF02089580959091FF028923E3
:1025B0008093FF0208951092FF0208958091DE0239
:1025C000089508950C94E1120C94E2129091A403E2
:1025D00092FD08C09091DE02981721F08093DE02F0
:1025E0000C94E41208958091DE02882329F0109261
:1025F000DE0280E00C94E4120895CF93DF93E09123
:102600000201F0910301809100038083E0910201B7
:10261000F091030190818091FF02892B808380914A
:10262000DE02882381F0E0910201F09103019081A4
:10263000892B808380910201909103010E949C2547
:1026400081110E94F312C0910201D091030140E276
:1026500050E06DEB72E0CE010E94792F892B69F07A
:1026600080E2FE01ADEBB2E001900D928A95E1F7B8
:10267000CE01DF91CF910C940D25DF91CF9108957C
:102680000C94E1129091A40392FD10C098E0899FF0
:1026900090011124262B2093DD020E94200E8091B0
:1026A000DD028595859585950C9440130C94200E3C
:1026B0001092DD0280E00C9440132091DD028095A1
:1026C00082238093DD02982F977099F430E0482F91
:1026D000082E000C550B2417350759F09091A403D0
:1026E00092FD07C08595859585950E94410E0C94B5
:1026F00058130895CF939091A40392FB222720F9B9
:102700002817F9F0C82F892FC0FB82F98093A40302
:102710008091A3039091A4030E94D61382E00E94AB
:102720005D138091290380FF0CC01F92CF9387EE29
:1027300092E09F938F930E949B070F900F900F90B2
:102740000F90CF9108958091A40382FB882780F990
:1027500091E089270C947A1381E00C947A1380E03D
:102760000C947A1380E090E00E948E2F21E0893E45
:102770009E4F09F020E0822F089582E090E00C94B3
:10278000862F83E090E00C94862FCF9384E090E036
:102790000E94862FC82F82E290E00E94862F2C2F65
:1027A00030E0A901582BCA01CF910895CF93C92FCA
:1027B000682F84E090E00E94942F6C2F82E290E0DA
:1027C000CF910C94942FAB01BC018FE090E00C945E
:1027D000A62FAB01BC0183E190E00C94A62F60E032
:1027E00070E0CB010C94E91360E070E0CB010E9433
:1027F000E3130C94EF1369EE7EEF80E090E00E940B
:10280000B22F60E082E090E00E94942F60E083E0CD
:1028100090E00E94942F10928102109282021092F6
:1028200083021092840260E084E090E00E94942F82
:1028300060E082E290E00E94942F60E085E090E00A
:102840000E94942F60E086E090E00E94942F6FEF4A
:1028500087E090E00E94942F40E050E0BA0188E0C9
:1028600090E00E94A62F60E08DE090E00E94942FFF
:1028700040E050E0BA0188E190E00E94A62F60E0BD
:1028800087E190E00E94942F40E050E0BA018CE193
:1028900090E00E94A62F60E070E080E290E00E944D
:1028A000B22F40E050E0BA0188E190E00E94A62FEC
:1028B0000C94F4130C94FB13682F8EE090E00C94AE
:1028C000942F0E94262760932503709326038093FC
:1028D000270390932803609321037093220380932E
:1028E000230390932403089585B7806885BF85B737
:1028F000806885BF089581E008950C947B14089545
:102900000C947F140C947F140C9482140C947F14F8
:102910000C9486140C947F140E9474148FE799E22F
:102920000E94F7240E948A140C9488140E94801438
:102930000C947F140E9475170C94DA080E941127DA
:102940000E94C3180E949A140E94C31E0C948414FF
:102950002F923F924F925F926F927F928F929F92AF
:10296000AF92BF92CF92DF92EF92FF920F931F939D
:10297000CF93DF93CDB7DEB72D970FB6F894DEBFB8
:102980000FBECDBF0E94D818282E81110E9461145D
:1029900081E093E09D878C8700E010E0302E802F4F
:1029A0000E9499172B013C01EC85FD858191919145
:1029B000A191B191FD87EC875301420188269926A8
:1029C000AA26BB2681149104A104B104B1F40F5FBF
:1029D0001F4F0830110511F78FEF89838A831B82FF
:1029E0000E941A278160782F9D838C8349815A81A8
:1029F0006B818D810E941D0951C08091290381FD49
:102A00000E94A5171B86C12CD12C7601C394D50139
:102A1000C4018C219D21AE21BF21892B8A2B8B2BB8
:102A200091F10E947D148823D1F0FB85FE833F82C3
:102A30004C205D206E207F2081E0452846284728D5
:102A400009F480E088870E941A278160782F9A878E
:102A500089874E815F8168858A850E941D09000FE4
:102A6000111F000F111FF801EF5FFC4F8081918152
:102A7000A281B381C826D926EA26FB26C082D1824C
:102A8000E282F3820BC08B858F5F8B87CC0CDD1CC1
:102A9000EE1CFF1C873109F0BACF99CF81E02110DD
:102AA00001C080E02D960FB6F894DEBF0FBECDBFFB
:102AB000DF91CF911F910F91FF90EF90DF90CF901A
:102AC000BF90AF909F908F907F906F905F904F904E
:102AD0003F902F9008950E94A8140E94631B0E94AB
:102AE000CE1D0C94EB08CF93DF930E949D16EC0152
:102AF000811521E5920708F045C0811530E593075F
:102B000008F094C0883E910528F5803E910508F0B4
:102B1000F8C0883A910570F4853A910508F07CC0B8
:102B20008130910509F475C008F4E8C0049708F0F5
:102B3000E8C0E4C08F3B910508F0E0C0C85AD0E07F
:102B4000CC0FDD1FC65BDE4F0990D881C02DCE01B2
:102B50009464D8C0811540E2940758F4811551E07F
:102B6000950708F0CEC08D3E910508F4C7C090656A
:102B7000C9C0C11580E4D80708F4C0C0DF70CE0119
:102B8000906AC0C0811525E59207A8F4811534E547
:102B9000930708F095C0811543E5940708F07BC0C2
:102BA000811552E5950708F061C0D82FCC27CE01DA
:102BB000816F906AA7C0C11589E5D807A0F4C11537
:102BC00028E5D20708F082C0C11536E5D30708F022
:102BD00095C08C2F0E9431178F7190E0D82FCC2791
:102BE000CE0190628FC0C1154AE5D40708F474C0C5
:102BF000CE0190568115904208F080C08D2F8F71C4
:102C00000E943117DD27D0628F71AE01582BCA01A7
:102C100079C081E090E076C0C55AD0E0C858DE4F58
:102C20008881C82FD0E0CE0190646CC074E0969586
:102C300087957A95E1F7282F23703C2F337081E038
:102C400090E002C0880F991F3A95E2F79C68AC01AA
:102C5000522B9A019C2F9F709695969550E2959FC6
:102C6000E0011124C9018C2B9D2B4CC08370992746
:102C700021E030E002C0220F331F8A95E2F79C2F3B
:102C80009695969580E2989FE0011124C22BD32B54
:102C9000CE019C6837C08370992721E030E002C0E4
:102CA000220F331F8A95E2F79C2F9695969540E266
:102CB000949FE0011124C22BD32BCE019A6822C02D
:102CC000D82FCC27CE01846F906A1CC0DC2FCC2774
:102CD000CE01806F906A16C08C2F8F700E943117C2
:102CE00094E0D695C7959A95E1F7CF70D0E0DC2FA8
:102CF000CC27D0699E01282BC90104C080E090E058
:102D000001C0CE01DF91CF91089528EB829FC001D1
:102D10001124FC0127E1729FE00DF11D1124E60F43
:102D2000F11DEE0FFF1FEE5BFE4F8591949108950C
:102D30000E9485160E94731508958238910569F1E5
:102D4000B0F48133910509F46DC048F489329105DE
:102D500009F463C08A32910509F469C00895853386
:102D6000910509F455C089339105B9F00895833E62
:102D7000910569F138F4803E9105B1F0823E9105EC
:102D800009F10895863E9105A9F1873E9105B9F1B3
:102D9000843E910509F064C023C02091A30320FD67
:102DA0004FC021FD4DC008958091A30380FD44C014
:102DB0008091A40380FF44C08091A30384FD42C09E
:102DC00083EE4DC08091A30382FF38C0F5CF809180
:102DD000A30382FD33C08091A40380FD31C0ECCFFA
:102DE0008091A40381FF32C08091A30384FD2AC097
:102DF00087EE35C08091A30383FF26C0F5CF809175
:102E0000A30383FD21C08091A40381FD1FC0ECCFEB
:102E10008091A30385FD1CC01DC08091A30385FD87
:102E200019C016C08091A30386FD16C017C08091FB
:102E3000A30386FD13C010C089E311C082EE0FC04A
:102E400080EE0DC080E00BC086EE09C084EE07C0A6
:102E500089E205C085E303C08AE201C081E390E016
:102E600008959091A30392FF0DC0282F2871283058
:102E700019F4877F846006C0282F2471243011F450
:102E80008B7F886093FF0DC0282F2871283119F49B
:102E9000877E846106C0282F2471243111F48B7E33
:102EA00088612091A40320FF0DC0382F387138307D
:102EB00019F4877F816006C0382F3171313011F4E9
:102EC0008E7F886021FF0DC0282F2871283119F4CA
:102ED000877E816106C0282F2171213111F48E7EF9
:102EE000886194FD877E089508950E94B213811130
:102EF00002C00E945A140E94BD13809329030E94AD
:102F0000C5139093A4038093A3030E9474170E9497
:102F1000C113682F70E080E090E00E94C00D6091C6
:102F20007D0270917E0280917F02909180020C94CC
:102F3000F80D24E0829FC0011124FC01EB53FC4FEB
:102F400060817181828193810895CF92DF92EF92A7
:102F5000FF920F931F93CF93DF938DE093E00E9436
:102F6000020785ECE82E83E0F82EC0E0D0E098E080
:102F7000C92E93E0D92E0EEF12E0DF93CF93DF92AC
:102F8000CF920E949B0785E093E00E940207F70121
:102F900061917191819191917F010E94A8089F9305
:102FA0008F937F936F931F930F930E949B078CEFD8
:102FB00092E00E94020721968DB79EB70A960FB63F
:102FC000F8949EBF0FBE8DBFC830D105B1F6DF911A
:102FD000CF911F910F91FF90EF90DF90CF900895C8
:102FE00080EA8A95F1F7089500C008950C94F017CF
:102FF00008950C94F8170C94F9170C94F8170C9486
:10300000FD17F894E82FE295EF70F0E031A1282F3A
:103010002F7081E090E001C0880F2A95EAF7982F81
:103020009095932391A392A1892B82A378940895DC
:103030000F931F93CF93DF93C2E9D1E089918F3F24
:1030400011F00E94011881E0CA39D807B9F7CBE71F
:10305000D1E002E911E089918F3F11F00E9401183F
:103060000C171D07C1F7DF91CF911F910F910895A4
:103070004F925F926F927F928F929F92AF92BF9288
:10308000DF92EF92FF920F931F93CF93DF938C0108
:10309000C62FD0E0CE018E569E4F7C01FC01908160
:1030A0009F3F09F460C0D62EF894E92FE295EF70A7
:1030B000F0E081A19F7021E030E001C0220F9A95DD
:1030C000EAF7822B81A382A12095282322A378945A
:1030D0000E94F417EBE7F1E022E931E0412C512C9A
:1030E00032014394812C912C540181918F3F99F0AE
:1030F000A82FA295AF70B0E090964C9150E08F70E1
:10310000BA0102C0759567958A95E2F760FD03C024
:10311000D301C20103C080E090E0DC01882A992A33
:10312000AA2ABB2A440C551C661C771C2E173F0785
:10313000E1F6F70180818F3F11F00E94011861E0F4
:1031400081149104A104B10409F460E08D2D0E9462
:10315000F617CC0FDD1FCC0FDD1FC00FD11F8882EB
:103160009982AA82BB82DF91CF911F910F91FF902C
:10317000EF90DF90BF90AF909F908F907F906F9077
:103180005F904F9008950E94181880E2E5ECF3E0FC
:10319000DF01982F1D929A95E9F7E5EAF3E0DF0148
:1031A0001D928A95E9F788E00E9423190C94F6078E
:1031B000FF920F931F93CF93DF93CDB7DEB7A09706
:1031C0000FB6F894DEBF0FBECDBF8E010F5F1F4F4D
:1031D00080E2F80111928A95E9F7F12C6F2DC80170
:1031E0000E943818F394F8E0FF12F8CF40E250E064
:1031F000B80185EA93E00E94792FFF24F3940097A9
:1032000009F4F12C892B41F080E2F801A5EAB3E042
:1032100001900D928A95E1F72F2D48E065EC73E05F
:1032200085EA93E00E9424190E94F8078F2DA0964A
:103230000FB6F894DEBF0FBECDBFDF91CF911F91C7
:103240000F91FF9008950895FF920F931F93CF93CE
:10325000DF93F82ED92F8B01C42F222349F081E070
:1032600080932C030E941A2790932B0380932A03A8
:1032700080912C038823F1F080912A0390912B03F5
:103280000E9432270597B0F0EF2DFD2FD80180E086
:1032900090E04C2F50E08417950754F40191119160
:1032A000219131910D931D932D933D930196F3CF71
:1032B00010922C03DF91CF911F910F91FF900895F1
:1032C0000E94FB290E949E140C94072A0E940B2A3C
:1032D0000E946B150C94292A0E94B8260E94E229AC
:1032E0000E948C140E9460190E9466190E94961414
:1032F000FBCF8091330380FF06C06091090170E02D
:10330000660F771F26C081FF04C06091090184E029
:1033100005C082FF07C06091090188E0689FB00185
:10332000112417C0909132039923D1F060910801C4
:10333000961788F72091090188E0289F90011124B1
:10334000929FA001939F500D112470E0CA010E942A
:10335000482F6038710540F46115710519F406C0F5
:1033600068E070E0862F08958FE7089581E0089562
:103370008091330380FF08C06091050170E075956E
:1033800067957595679521C081FF06C0609105011D
:1033900070E07595679519C082FF04C060910501C2
:1033A00070E010C090913103992399F0609104016D
:1033B0009617A0F780910501899FC001112470E044
:1033C0000E94482F6038710540F46115710519F4A9
:1033D00006C061E070E0862F08958FE7089581E0D0
:1033E00008958D3E21F40E947919819504C08E3E86
:1033F00029F40E9479198093370308958F3E21F4B0
:103400000E947919819504C0803F29F40E9479199E
:10341000809336030895893F19F40E94B81905C0B6
:103420008A3F31F40E94B81981958093380308953A
:103430008B3F21F40E94B819819504C08C3F29F478
:103440000E94B8198093390308959FE0980F98302F
:1034500078F421E030E0A90102C0440F551F9A958D
:10346000E2F7CA0190913503892B809335030895C3
:103470008D3F21F48091330381600BC08E3F21F496
:1034800080913303826005C08F3F29F4809133031C
:1034900084608093330308958D3E39F4909137030F
:1034A00097FF35C01092370359C08E3E29F4909192
:1034B00037031916BCF32BC0909136038F3E29F4C5
:1034C00097FF25C01092360349C0803F19F41916A2
:1034D000CCF31DC090913803893F29F41916BCF430
:1034E000109238033BC08A3F19F497FF10C0F8CF01
:1034F0008B3F39F49091390397FF09C0109239033B
:103500002DC08C3F21F4909139031916BCF39FE034
:10351000980F983080F421E030E0A90102C0440FF8
:10352000551F9A95E2F7CA0180959091350389233A
:103530008093350313C08D3F21F4809133038E7F38
:103540000BC08E3F21F4809133038D7F05C08F3FE8
:1035500029F4809133038B7F80933303809136036A
:10356000811106C080913703811102C0109232038D
:1035700080913803811106C080913903811102C006
:103580001092310308958091290383FF7EC08BE55B
:1035900093E00E940207809135031F928F9386E586
:1035A00093E09F938F930E949B0784E593E00E9492
:1035B000020780913603282F082E000C330B3F930F
:1035C0008F9381E593E09F938F930E949B078FE4F5
:1035D00093E00E94020780913703282F082E000CE9
:1035E000330B3F938F938CE493E09F938F930E94D0
:1035F0009B078AE493E00E94020780913803282FFA
:10360000082E000C330B3F938F9387E493E09F9336
:103610008F930E949B0785E493E00E9402078091AC
:103620003903282F082E000C330B3F938F9382E42D
:1036300093E09F938F930E949B078FE393E00E94F8
:103640000207809132031F928F938CE393E09F9344
:103650008F930E949B078AE393E00E940207809168
:1036600033031F928F9387E393E09F938F930E947E
:103670009B0784E393E00E9402078DB79EB74C96A8
:103680000FB6F8949EBF0FBE8DBF0E941A272091DF
:103690003603211104C020913703222321F0909397
:1036A000300380932F0320913803211104C020910F
:1036B0003903222321F090932E0380932D0384E37A
:1036C00093E00C946225EF92FF920F931F93CF9398
:1036D000DF9300D000D000D0CDB7DEB786E0E4E3C2
:1036E000F3E0DE01119601900D928A95E1F7E090EA
:1036F0003603F0903703009138031091390310928C
:103700003603109237031092380310923903E110F8
:1037100003C0FF2009F45DC080912F039091300316
:103720000E943227AC0190913203992339F0209105
:103730000A0130E02417350758F04BC020910B01E7
:103740008AE0289F900111242417350718F041C002
:103750009F3F19F09F5F90933203EE2061F00E942B
:1037600079191E1414F09FEF01C091E0989F902DDD
:10377000112490933603FF2061F00E9479191F14E1
:1037800014F09FEF01C091E0989F902D1124909329
:103790003703309136033323E1F02091370322239E
:1037A000C1F045EB3403C0011124992319F0909323
:1037B000360303C081E08093360335EB2303C00159
:1037C0001124992319F09093370303C081E080936B
:1037D0003703011103C0112309F45DC080912D034B
:1037E00090912E030E943227AC01909131039923CE
:1037F00039F02091060130E02417350758F04BC00E
:10380000209107018AE0289F900111242417350791
:1038100018F041C09F3F19F09F5F90933103002340
:1038200061F00E94B819101614F09FEF01C091E0EA
:10383000989F902D112490933803112361F00E94DA
:10384000B819111614F09FEF01C091E0989F902DC8
:10385000112490933903309138033323E1F0209100
:1038600039032223C1F045EB3403C001112499230D
:1038700019F09093380303C081E08093380335EB4F
:103880002303C0011124992319F09093390303C035
:1038900081E0809339038091360381110BC08091C0
:1038A0003703811107C080913803811103C08091D3
:1038B000390381110E94C31AEB82FC820D831E839F
:1038C00086E0FE013196A4E3B3E001900D928A9563
:1038D000E1F726960FB6F894DEBF0FBECDBFDF919D
:1038E000CF911F910F91FF90EF900895E4E3F3E0E3
:1038F00086E0DF011D928A95E9F71092320310925B
:103900003103109233030895CF93DF93EC01FB0151
:103910008281882309F43CC1C430FDE5DF0760F4EF
:10392000CB3F9CE5D90788F49E0122503C452431C9
:10393000310508F02EC109C0C236EDE5DE0729F0D9
:10394000C63AFDE5DF0709F024C10E94C513909334
:10395000A4038093A303C1318CE5D80709F4C6C042
:1039600008F042C0C930ECE5DE0709F49BC000F561
:10397000C5308CE5D80709F485C078F4C330ECE590
:10398000DE0709F478C008F07AC0C230DC4509F0DF
:10399000F5C08091A3038160EFC0C7309CE5D907D3
:1039A00009F478C008F07AC08091A3038061E4C074
:1039B000CD30FCE5DF0709F487C058F4CB309CE537
:1039C000D90709F479C008F07BC08091A30388600F
:1039D0006FC0CF30FCE5DF0709F480C008F082C07B
:1039E0008091A303877FC8C0CE3F9CE5D90709F427
:1039F00071C000F5C531FCE5DF0709F485C068F446
:103A0000C3319CE5D90709F475C008F095C00E9440
:103A1000680D8091A3038F77AFC0CC3FFCE5DF0733
:103A2000A9F108F054C0CB3FDC4509F0A7C0809154
:103A3000A40340C0C230EDE5DE0709F489C058F4A4
:103A4000C1158DE5D80709F45AC008F069C0809106
:103A5000A40382602FC0C236EDE5DE0709F47CC006
:103A6000C63AFDE5DF0709F481C0C330DD4509F042
:103A700085C080E06EC08091A30382607DC080918C
:103A8000A30316C08091A303886076C08091A4032D
:103A900082604FC08091A30380626EC08091A303B7
:103AA00080646AC00E94680D8091A303806864C02E
:103AB000846062C081603DC08091A3038E7F5CC042
:103AC0008091A3038D7F58C08091A30316C080917D
:103AD000A40318C08091A4038D7F2BC08091A30301
:103AE0008F7E4AC08091A3038F7D46C08091A3033F
:103AF0008F7B42C08091A303877F8B7F3DC08091E5
:103B0000A4038D7F8E7F15C08091A30382FB2227A3
:103B100020F991E0922790FB82F990FB83F92CC069
:103B20008091A403982F909591708E7F892B90FBA4
:103B300081F98093A40322C00E94680D8091A303A1
:103B400087FB222720F991E0922790FB87F914C088
:103B500081E00E945C1412C08091A30384FB2227A1
:103B600020F991E0922790FB84F906C08091A3038D
:103B7000982F909590FB80F98093A3038091A303E5
:103B80009091A4030E94D6130E94680D80E001C0AA
:103B900081E0DF91CF910895089508958BEE0E9402
:103BA000971F8A3FA1F40E94821F9091A103892B45
:103BB00080933F030E94821F809340030E94821FD4
:103BC0009091400320913F03992349F014C08091C4
:103BD000290383FFB1C084EC93E00C9402078111A8
:103BE0000AC030914203311106C030913D033227A3
:103BF000377009F497C020933D03322F307424FFAF
:103C000007C031110AC0903841F097FD09C005C0C6
:103C1000311105C097FF04C002C091E801C09FE7C1
:103C20009093400325FF07C027FD0AC0803841F06C
:103C300087FD09C005C027FD05C087FF04C002C07D
:103C400081E801C08FE7922F977090933F03819591
:103C50008093410380913C0322FF27C0811109C05A
:103C60000E941A2790933B0380933A0381E080934C
:103C70003C039091400380914103911102C088233D
:103C8000C1F122E020933C0387FD8F5F85958195EC
:103C900080934203892F97FD8F5F8595809343031F
:103CA000109240031092410324C0813001F58091AD
:103CB0003A0390913B030E9432278C329140B8F432
:103CC00080913F03846080933F038EE393E00E94E2
:103CD00062258FEF91EE24E0815090402040E1F783
:103CE00000C0000080913F038B7F80933F031092C0
:103CF0003C0380913F038B7F80933F03809140037F
:103D0000811108C080914103811104C08091420358
:103D1000882321F08EE393E00E94CD1D8EE393E093
:103D20000E946225109240031092410310924203B8
:103D30001092430310923F030895CF9384EF0E94A3
:103D4000971FC82F8091290383FF1BC084EA93E04B
:103D50000E940207809166031F928F931F92CF9358
:103D60001F9284EF8F938EE793E09F938F930E942F
:103D70009B078DB79EB708960FB6F8949EBF0FBEEF
:103D80008DBFCF910895CF930E946F1F2FEF83EDCA
:103D900090E3215080409040E1F700C000008FEF99
:103DA0000E94971FC82F8091290383FF1BC085E7BE
:103DB00094E00E940207809166031F928F931F92E6
:103DC000CF931F928FEF8F938FE494E09F938F9305
:103DD0000E949B078DB79EB708960FB6F8949EBFBA
:103DE0000FBE8DBF0E94821FC82F8091290383FFC1
:103DF00016C086E394E00E940207809166031F923A
:103E00008F931F92CF938DE194E09F938F930E94A5
:103E10009B070F900F900F900F900F900F900E94A4
:103E2000821FC82F8091290383FF16C082E094E08F
:103E30000E940207809166031F928F931F92CF9377
:103E400089EE93E09F938F930E949B070F900F90B2
:103E50000F900F900F900F900E949D1ECF910C9489
:103E6000CC1D9FB7F894209144038091450382179D
:103E700061F030E0F901EA5BFC4F80812F5F3F4F3A
:103E80002F7133272093440301C080E09FBF089522
:103E9000CF93DF93EC010E94CA20882341F0209742
:103EA00031F085E08A95F1F700002197F4CFCE013B
:103EB000DF91CF910895CF93DF93C2E3D0E00E94CA
:103EC000CA20811108C0209731F085E08A95F1F76A
:103ED00000002197F4CFCE01DF91CF9108950E9489
:103EE000C7200E94D8205D985A9886E78093CA0020
:103EF0001092C8001092CD001092CC0080E98093FF
:103F0000C90008958AE1815011F40C94311F3FB724
:103F1000F89420914503909144033FBF2913F5CFB6
:103F2000EFE9FFE03197F1F700C00000ECCFEF922E
:103F3000FF920F931F93CF93DF93E82E10926603A7
:103F40001092CA008091C900877E8093C9000E94A8
:103F5000C4200E94D8208FE891E00197F1F700C0BB
:103F600000000E94D5200E94C72080E197E20E94B5
:103F7000481F892B11F48AE077C0C0E0D0E011E03F
:103F8000F12C01E090E59A95F1F7C7010C2E02C0E3
:103F9000959587950A94E2F780FF04C010270E9448
:103FA000D82002C00E94D5200E945B1F892B11F4EB
:103FB00082E05AC082E390E00E94481F892B11F4EE
:103FC00083E052C02196C830D105E1F680E58A959C
:103FD000F1F7112319F00E94D82002C00E94D520C9
:103FE0000E945B1F892B11F484E03EC082E390E0C5
:103FF0000E94481F892B11F485E036C090E59A9500
:10400000F1F70E94D820C2E3D0E00E94DB20882391
:1040100041F0209741F025E02A95F1F70000219723
:10402000F4CFCD2B11F486E01FC082E390E00E9414
:10403000481F892B11F487E017C00E945B1F892B52
:1040400019F0C2E3D0E009C088E00EC0209759F013
:1040500085E08A95F1F7000021970E94DB208823F4
:10406000A9F3CD2BE9F489E0809366030E94C72071
:104070000E94D8205D985A9886E78093CA001092D3
:10408000C8001092CD001092CC0080E98093C90046
:1040900080E0DF91CF911F910F91FF90EF900895F5
:1040A0000E94C7200E94D8205D985A9886E7809386
:1040B000CA001092C8001092CD001092CC0080E986
:1040C0008093C900DF91CF911F910F91FF90EF90E6
:1040D0000C94821F1F920F920FB60F9211240BB6F1
:1040E0000F922F933F934F935F936F937F938F9391
:1040F0009F93AF93BF93CF93EF93FF938091C800AB
:104100008C714091CE0081111BC0CFB7F894809183
:10411000450390E09C012F5F3F4F2F713327509153
:104120004403521739F0FC01EA5BFC4F40832093B3
:10413000450304C083E994E00E940207CFBF10C08A
:104140001F924F931F928F938FE994E09F938F93C9
:104150000E949B070F900F900F900F900F900F9061
:10416000FF91EF91CF91BF91AF919F918F917F91EF
:104170006F915F914F913F912F910F900BBE0F90D8
:104180000FBE0F901F9018955D98559A08955598F9
:104190005D9A089555985D9A85E08A95F1F700003B
:1041A00089B185FB882780F908955A98529A089515
:1041B00052985A9A089552985A9A85E08A95F1F73A
:1041C000000089B182FB882780F90895809104015D
:1041D0001F928F93809105011F928F938091080108
:1041E0001F928F93809109011F928F9380910A01F2
:1041F0001F928F9380910B011F928F9381EC94E01B
:104200009F938F930E949B078DB79EB70E960FB614
:10421000F8949EBF0FBE8DBF0895883220F58E3171
:1042200008F068C08B3091F1C0F4873009F0BEC04F
:1042300081E080930B0184E180930A018AE08093FE
:1042400009018EE18093080188E08093050188E2EE
:104250008093040183E296E0C6C0833109F443C031
:10426000843169F1A3C08F3409F49EC028F48932E7
:1042700031F1883359F09AC0813531F008F4D4C057
:10428000823509F4A7C092C08FEFA5C085E496E0FF
:104290000E9402070E94E6201F9281E08F931F92E6
:1042A00088E08F938EE395E09F938F930E949B0706
:1042B0000F900F900F900F900F900F9096C082E488
:1042C00096E00E94020780916B03882309F4AAC03C
:1042D00010926B0310926A031092690310926803A4
:1042E00010926703B1C084E396E00E9402070E9427
:1042F000E6207BC08D5180936B03833031F170F4E5
:104300008130D1F0823009F03FC08AE091E0909393
:104310006A038093690387EA91E01FC0853059F1F1
:1043200008F1863089F584E091E090936A038093E8
:10433000690382EE91E011C08BE091E090936A03F3
:10434000809369038EE991E008C089E091E0909341
:104350006A038093690383EB91E0909368038093F1
:10436000670318C088E091E090936A038093690323
:1043700080EC91E0F2CF85E091E090936A03809326
:1043800069038FEC91E0E9CF10926B0381E396E033
:104390000E94020780916B03882309F455C01F9285
:1043A0008F938DE296E00DC08AE015C080E296E022
:1043B0001AC097FF47C0108280811F928F938AE1B5
:1043C00096E09F938F930E949B070F900F900F9002
:1043D0000F900BC081E0E0916903F0916A03309780
:1043E00029F587E196E00E94020720916B032223C2
:1043F00059F18091670390916803009711F48AE95D
:1044000091E09F938F931F922F938EE096E09F935E
:104410008F930E949B070F900F900F900F900F901B
:104420000F9016C080E0089586EFD5CF2081082E2A
:10443000000C990B820F911D8F3F910509F00CF430
:10444000B8CF8FEF8083B8CF8AE096E00E94020752
:1044500081E00895CF93C82F1F928F938BE596E04C
:104460009F938F930E949B0781E090E0A0E0B0E0D3
:10447000BC01CD0104C0660F771F881F991FCA9524
:10448000D2F70E94C00D0F900F900F900F90CF9118
:104490000C94680DDF92EF92FF920F931F93CF93CE
:1044A000DF93482F50E0FA013597EF33F10508F01C
:1044B0003FC1E85AFF4F0C945C2F0E94C1131F921A
:1044C0008F9381EB9AE09F938F930E949B070E94AA
:1044D000BD1383FB992790F91F929F9382FB992725
:1044E00090F91F929F9381FB992790F91F929F93B8
:1044F000982F91701F929F931F928F9388E69AE056
:104500009F938F930E949B070E94C51387FB2227CE
:1045100020F91F922F9386FB222720F91F922F93B9
:1045200085FB222720F91F922F9384FB222720F955
:104530001F922F9383FB222720F91F922F9382FB38
:10454000222720F91F922F9391FB222720F91F92F7
:104550002F93292F21701F922F9381FB222720F95F
:104560001F922F93282F21701F922F939F938F9329
:1045700083E899E09F938F930E949B078DB79EB726
:1045800088960FB6F8949EBF0FBE8DBF06C081E718
:104590009BE00E9402070E945A14C1E0CEC081ED48
:1045A00097E074C080912903817F8E7F80932903D7
:1045B0008AEA97E00E9402078DE69BE00E940207CC
:1045C00081E080936C03E9CF81E59BE00E940207C4
:1045D0000E94FB07E2CF80912903C82FC095C170CC
:1045E000C0FB80F980932903CC2319F085E49BE07C
:1045F00091C088E39BE00E94020780912903897F94
:10460000877F80932903C9CF9091290391FBCC2701
:10461000C0F981E0C827892FC0FB81F98093290365
:10462000CC2319F08BE29BE027C08DE19BE02EC0EC
:104630009091290392FBCC27C0F981E0C827892FEC
:10464000C0FB82F980932903CC2319F08EE09BE014
:1046500013C08EEF9AE01AC09091290393FBCC27E8
:10466000C0F981E0C827892FC0FB83F98093290313
:10467000CC2351F082EF9AE00E9402078091290337
:1046800081608093290359C085EE9AE00E94020759
:1046900084CF84EE96E0FACF0E942627062FF72ECD
:1046A000E82ED92EC091A303C7FBCC27C0F91091E7
:1046B000A003D09118010E940125DF92EF92FF9292
:1046C0000F931F92CF931F921F931F92DF931F92FE
:1046D0008F9380E696E09F938F930E949B078DB700
:1046E0009EB70E960FB6F8949EBF0FBE8DBF55CFE6
:1046F0000E94680D9091A30397FBCC27C0F981E03D
:10470000C827892FC0FB87F98093A303CC2329F006
:104710008BED9AE00E94020710C080ED9AE0B6CFC0
:10472000895303C08D5101C080E00E942A2235CFF9
:104730008EEC9AE00E940207C0E08C2FDF91CF91AF
:104740001F910F91FF90EF90DF90089580E0089502
:104750000C94A623CF93C82F80916C03813071F005
:1047600040F0823009F045C08C2F0E940D2181E07D
:1047700046C00E94BB128232F1F504C00E94BB12F7
:10478000823261F48C2F0E94A823811104C08C2FE7
:104790000E944A222CC081E090E029C08C2F0E9408
:1047A000A623811123C0C431C9F058F4CB3069F07D
:1047B000C031B9F482E080936C0388E30E940D213C
:1047C00015C0C93259F0C83361F48AEA97E00E94F3
:1047D000020787E596E00E94020708C010926C036A
:1047E0000CC085E596E00E94020707C081E0817059
:1047F00006C010926C0380E002C080E0F8CFCF9139
:104800000895CF93DF9386319C4541F5EB010E94DB
:10481000BB12982F8A8120910201309103018823D5
:1048200079F09A7A81E009F480E080936D03911128
:1048300002C069E201C065E3C9010E9454260AC0B2
:1048400080916D03811102C069E201C065E3C90175
:104850000E945F260E94FD1280E001C081E0DF918E
:10486000CF9108950F931F93CF93DF93C42FD22F2F
:10487000FC0182818823C9F0409370030E941A27AB
:1048800090936F0380936E0380E28C0F883008F062
:1048900057C0C77081E001C0880FCA95EAF7DF9161
:1048A000CF911F910F910C94B70A80917003481318
:1048B00030C080916E0390916F030E943227883C34
:1048C000910538F510E21D0FCD17B9F080E28C0F7D
:1048D000883040F4C77081E001C0880FCA95EAF7BC
:1048E0000E94BE0A183028F581E09D2F977001C004
:1048F000880F9A95EAF70E94B70A802F0E94AE0AA5
:104900001830F0F4D77081E001C0880FDA95EAF72B
:104910000AC080E28C0F883098F4C77081E001C033
:10492000880FCA95EAF7DF91CF911F910F910C94F0
:10493000BE0A802FDF91CF911F910F910C94AE0A88
:10494000DF91CF911F910F9108950F939C01CB019F
:10495000243F4CE5340731F188F4293DFCE53F075D
:10496000D9F02A3D4CE5340779F1283D3C45A9F5BD
:1049700006E221EE41EE68ED7CE52BC0263FFCE52A
:104980003F07E1F0A8F0273F3C4539F507E225EE67
:1049900046EE67EF7CE51DC007E225EE45EE69EDCA
:1049A0007CE517C006E221EE40EE64EF7CE511C025
:1049B00007E225EE44EE65EF7CE50BC006E221EE52
:1049C00042EE66EF7CE505C008E221E045EE6AEDC7
:1049D0007CE50E94322480E008C0FC0182818823AB
:1049E00019F01092700301C081E00F910895909327
:1049F00007028093060208959093760380937503CF
:104A00000895E0917503F0917603309721F00190BD
:104A1000F081E02D099480E00895EF92FF921F93BA
:104A2000CF93DF93FC01A0917503B09176031097AB
:104A300009F442C080911801882341F08091A303BA
:104A400087FF04C08081818386E08083EF01129616
:104A5000ED91FC911397CE0109958091290382FF76
:104A60002BC080FF04C08AE89BE00E94020718E088
:104A700084E8E82E8BE0F82E8091290380FF0BC09C
:104A800088811F928F93FF92EF920E949B070F9055
:104A90000F900F900F90115021961111EDCF809132
:104AA000290380FF09C082E89BE0DF91CF911F912D
:104AB000FF90EF900C940207DF91CF911F91FF9030
:104AC000EF900895E0917503F0917603309739F0F7
:104AD00022E0DC012C930480F581E02D09940895F7
:104AE00020917303309174032817390771F0909364
:104AF000740380937303E0917503F091760330970C
:104B000021F00680F781E02D09940895209171032A
:104B1000309172032817390771F0909372038093D4
:104B20007103E0917503F0917603309721F00084D2
:104B3000F185E02D09940895FC01329680911801C9
:104B4000882331F08091A30387FF02C09EE101C05A
:104B500096E080E0915028F021912223D9F38F5FD5
:104B6000F9CF0895662351F1209118012223E9F02D
:104B70002091A30327FF19C0462F469546954695D9
:104B80004E31E0F4677021E030E002C0220F331FA5
:104B90006A95E2F7FC01E40FF11D828190E0282381
:104BA000392381E0232B69F409C0FC013296089671
:104BB0002191621729F0E817F907D1F780E00895ED
:104BC00081E008959C01FC0132969FEF80E04191C5
:104BD000461789F09F3F19F4411101C0982F8F5F4C
:104BE0008630A9F79F3F39F0F901E90FF11D97FDD4
:104BF000FA956283089508959C012A5F3F4FFC0156
:104C00004281461301C01282019682179307B9F7B9
:104C10000895262F2695269526952E3170F4FC01B1
:104C2000E20FF11D677021E030E001C0220F6A95AC
:104C3000EAF78281282B228308958091290380FF3F
:104C40000CC01F926F938AEB9BE09F938F930E94FF
:104C50009B070F900F900F900F900895262F269589
:104C6000269526952E3178F4FC01E20FF11D677030
:104C700021E030E001C0220F6A95EAF72095828199
:104C80002823228308958091290380FF0CC01F925E
:104C90006F938CE99BE09F938F930E949B070F90EB
:104CA0000F900F900F90089520911801222329F062
:104CB0002091A30327FD0C9409260C94E225209152
:104CC0001801222329F02091A30327FD0C942E26FE
:104CD0000C94FC2520911801FC013296222331F01E
:104CE0008091A30387FF02C08EE101C086E0DF014F
:104CF0001D928A95E9F7089508950C947C2683E027
:104D0000809377030C947D26811102C081E001C05D
:104D100082E0809377030C947D260C94842681E0B6
:104D2000809377030C947D260C948F2608950C9421
:104D300096260C9497260C9496260C9496260C9402
:104D40009626CF930E949D260E94D8180E949B26EB
:104D5000C0E08C2F0E949917672B682B692B29F4D0
:104D6000CF5FC830B1F780E001C081E0CF910895F6
:104D700008951F920F920FB60F9211248F939F9355
:104D8000AF93BF9380917803811113C08091E503A5
:104D90009091E603A091E703B091E8034196A11D2D
:104DA000B11D8093E5039093E603A093E703B093CE
:104DB000E803BF91AF919F918F910F900FBE0F901D
:104DC0001F9018958091ED03843031F10E947B088B
:104DD0001092780320E488E190E00FB6F894A8954B
:104DE000809360000FBE2093600083B7817F846052
:104DF00083BF83B7816083BF7894889583B78E7FA4
:104E000083BF0FB6F894A895809160008861809365
:104E10006000109260000FBE08950E94680D0C940F
:104E20007F0882E084BD93E095BD9AEF97BD8093A3
:104E30006E0008952FB7F8948091E5039091E603F2
:104E4000A091E703B091E8032FBF08952FB7F8941E
:104E50006091E5037091E6038091E7039091E80388
:104E60002FBF08959C014FB7F8948091E50390916E
:104E7000E603A091E703B091E8034FBF821B930BB9
:104E8000089578941F920F920FB60F9211248F936A
:104E90009F93AF93BF938091E5039091E603A09118
:104EA000E703B091E8030196A11DB11D8093E503CE
:104EB0009093E603A093E703B093E803BF91AF910B
:104EC0009F918F910F900FBE0F901F901895F8949F
:104ED00081E08093E00080E28093D800E9ECF0E08C
:104EE00010828FE19EE40197F1F700C000001DBA27
:104EF000109268001CBC10BE1FBA10927A0010926B
:104F00006E0010926F00109270001092710010826B
:104F10001092BC0011B814B817B81AB81DB810BA5E
:104F200012B815B818B81BB81EB811BA0C9400FE08
:104F3000089580919F030895089522E02093E90049
:104F40002FEF3091E800215035FD06C035ED3A9540
:104F5000F1F700002111F5CF2091E80025FF0BC0EB
:104F600040E050E066E070E00E94982A8091E800FE
:104F70008E778093E8000895CF93DF9320911801F6
:104F8000222339F02091A30327FF03C060E222E02F
:104F900002C068E021E02093E9002FEF3091E800A3
:104FA000215035FD06C035ED3A95F1F7000021118D
:104FB000F5CF2091E80025FF1DC0EC01809118017C
:104FC000811105C040E050E068E070E003C070E08F
:104FD00040E050E0CE010E94982A8091E8008E7750
:104FE0008093E80080E2FE01AFE7B3E001900D920C
:104FF0008A95E1F7DF91CF91089580937B037093B9
:105000007D0360937C038091ED03843001F582E0A1
:105010008093E9008FEF9091E800815095FD06C0E4
:1050200095ED9A95F1F700008111F5CF8091E80098
:1050300085FF0DC040E050E063E070E08BE793E057
:105040000E94982A8091E8008E778093E800089566
:10505000BC0184E00C94FD27BC0183E00C94FD2787
:105060008CEE9BE00E9402078091EC03811109C045
:105070000E94252C0E94872C8091E20084608093FE
:10508000E200089588EE9BE00E9402071092EC0374
:10509000089584EE9BE00E9402070C94942680EE13
:1050A0009BE00E9402076091E90381E0611101C069
:1050B00080E00C947F268CED9BE00E94020790918B
:1050C000ED0381E0943009F080E06091E9030C94F5
:1050D000842620917A032F5F822F62E30E943C2F67
:1050E000992319F020937A03089510927A038091FE
:1050F0007E03882371F18091ED03843041F5809126
:10510000E9008F702091EC00922F917020FD90E8C3
:10511000892B93E09093E9009091EB0090FF14C0ED
:105120009091EE0097FF10C09091E80095FF03C0AA
:105130001092F100F9CF9091E80090FF05C0909196
:10514000E8009E779093E8008F708093E9001092BA
:105150007E03089542E061EC81E00E949E2B42E2D2
:1051600061EC82E00E949E2B42E261EC83E00E94AF
:105170009E2B9091ED0381E0943009F080E06091E6
:10518000E9030C948D268091EF03833009F45FC00E
:1051900030F4813071F0823009F498C008958A307B
:1051A00009F484C08B3009F46AC0893009F0A6C0C4
:1051B00020C08091EE03813A09F0A0C08091E80000
:1051C000877F8093E8008091F2039091F303892B0D
:1051D00021F460E28FE793E003C060E080E090E0BC
:1051E00070E00E94E32A8091E8008B778093E800CA
:1051F00008958091EE03813209F080C08091F2031E
:105200009091F303029708F079C08091E800877FBE
:105210008093E8008091E80082FD05C08091ED0355
:105220008111F8CF6BC08091F2009091F30002974A
:1052300031F48091F100813011F0863021F48091B9
:10524000F10080939F038091E8008B7753C0809199
:10525000EE03813A09F052C08091F2039091F3037A
:10526000892B09F04BC08091E800877F8093E8008C
:105270008091E80080FFFCCF8091180136C08091BA
:10528000EE038132D9F58091F2039091F303892BDB
:10529000A9F58091E800877F8093E8000E94D32BD6
:1052A0008091F003809318010C94680D8091EE03B7
:1052B000813221F58091E800877F8093E8000E9489
:1052C000D32B8091F1038093A00308958091EE0386
:1052D000813AA1F48091E800877F8093E800809173
:1052E000E80080FFFCCF8091A0038093F1008091C3
:1052F000E8008E778093E8000C94D32B08959FB735
:10530000F89410927E039FBF9091ED03943009F0C2
:1053100057C09091E9009F703091EC00232F2170CD
:1053200030FD20E8922B23E02093E9002091EB0050
:1053300020FF43C02091EE0027FF3FC0209179035A
:10534000222321F02091E80025FF37C01092790335
:1053500026E03091E80035FD15C03091ED03343082
:1053600061F53091EB0035FD28C0215021F481E03A
:105370008093790322C0EFE9FFE03197F1F700C095
:105380000000E7CF8093F1008091E80085FD0AC01E
:105390008091E80080FFFCCF8091E8008E778093B9
:1053A000E80006C08FB7F89421E020937E038FBFFA
:1053B0009F709093E90080E008959F709093E900BA
:1053C0008FEF089584B7877F84BF0FB6F894A895B0
:1053D00080916000886180936000109260000FBE31
:1053E00090E080E80FB6F89480936100909361009C
:1053F0000FBE0C948F260E94252C0E94872CE2EE73
:10540000F0E080818460808378940C94212F8CE07C
:1054100091E00C94FC248091ED038530C9F488ED73
:105420009BE00E9402078091ED03853079F40E9491
:10543000E2268091EB038823B1F30E94A126882302
:1054400091F30E94822A0E94680DEDCF0C940D27E3
:10545000089508950C942C2A292F332723303105E1
:10546000C9F060F42130310581F02230310509F0B6
:1054700041C08BE590E024E23CE040C021323105A0
:10548000E1F02232310531F135C082E190E02FE7C1
:105490003CE034C099278130910549F028F002970B
:1054A00049F5E0EFFBE005C0E0E2FCE002C0E6E128
:1054B000FCE0849190E09F0121C063307105D0F43D
:1054C000660F771FFB01E050FE4F2081318189E09C
:1054D00090E014C06330710568F4FB01EE0FFF1F0C
:1054E000E650FE4F20813181FB01E950FE4F808163
:1054F00090E004C080E090E020E030E0FA013183E9
:105500002083089584E189BD86E189BD09B400FE48
:10551000FDCF8091D8008F7D8093D8008091E000EE
:1055200082608093E0008091E00081FDFCCF0895CF
:10553000CF92DF92EF92FF920F931F93CF93DF935F
:10554000EC018B017A010E94F22B811133C0E1142E
:10555000F10439F0F70180819181081B190BC80F04
:10556000D91FC12CD12C0115110519F18091E8002A
:1055700085FD16C08091E8008E778093E800E114E5
:10558000F10449F0F70180819181C80ED91ED182C2
:10559000C08285E00FC00E94F22B882321F30AC04D
:1055A00089918093F10001501109FFEFCF1ADF0AB2
:1055B000DACF80E0DF91CF911F910F91FF90EF90B4
:1055C000DF90CF9008952091F4033091F5032617D2
:1055D000370748F06115710539F42091E8002E77FE
:1055E0002093E80001C0B901FC0120E061157105BC
:1055F00069F18091ED038823E1F18530E1F180913B
:10560000E80083FD3AC08091E80082FD2CC08091C3
:10561000E80080FFEBCF8091F2009091F3006115DC
:10562000710551F08830910538F421912093F100F3
:10563000615071090196F3CF21E0089709F020E04D
:105640008091E8008E778093E800D0CF2111D1CFF0
:105650000AC08091ED03882361F0853061F080916C
:10566000E80083FD0AC08091E80082FFF2CF80E06D
:10567000089582E0089583E0089581E008952091DF
:10568000F4033091F5032617370748F061157105CB
:1056900039F42091E8002E772093E80001C0B90189
:1056A000FC0120E06115710581F18091ED038823F3
:1056B00009F43EC0853009F43DC08091E80083FDC7
:1056C0003BC08091E80082FD2DC08091E80080FF02
:1056D000E9CF8091F2009091F3006115710559F0C6
:1056E0008830910540F424912093F1003196615067
:1056F00071090196F2CF21E0089709F020E080912E
:10570000E8008E778093E800CDCF2111CECF0AC07C
:105710008091ED03882361F0853061F08091E8008D
:1057200083FD0AC08091E80082FFF2CF80E00895F7
:1057300082E0089583E0089581E00895982F9730DE
:1057400068F59093E900981739F07091EC0020917A
:10575000ED005091F00003C0242F762F50E021FD82
:1057600002C09F5FECCF3091EB003E7F3093EB00A7
:105770003091ED003D7F3093ED003091EB003160D2
:105780003093EB007093EC002093ED005093F00009
:105790002091EE0027FDE5CF80E008958F70809383
:1057A000E90081E008958091EE0387FF11C08091A8
:1057B000E80082FD05C08091ED038111F8CF11C092
:1057C0008091E8008B770BC08091ED03882349F02E
:1057D0008091E80080FFF8CF8091E8008E77809379
:1057E000E80008952091E4003091E50095E64091AD
:1057F000EC00842F817040FF23C08091E80080FD81
:105800001DC08091ED03882399F0853099F0809137
:10581000EB0085FD11C04091E4005091E500241794
:10582000350729F3915011F09A01E1CF84E00895F2
:1058300082E0089583E0089581E0089580E008956E
:105840004091E80042FFDDCF08950E94962C0E940F
:105850009E2CE0EEF0E0808181608083E8EDF0E056
:1058600080818F77808319BCA7EDB0E08C918E7F0B
:105870008C9380818F7E80831092EC0308950F9328
:105880001F93CF93DF930E94962C0E949E2CC8ED0D
:10589000D0E088818F778883888180688883888139
:1058A0008F7D8883E7EDF0E080818068808319BC7C
:1058B0001092ED031092E9031092EB031092EA03A9
:1058C00000EE10E0F80180818B7F80838881816009
:1058D000888342E060E080E00E949E2BE1EEF0E0F1
:1058E00080818E7F8083E2EEF0E080818160808322
:1058F000808188608083F80180818E7F80838881A9
:1059000080618883DF91CF911F910F910895E8ED19
:10591000F0E080818F7E8083E7EDF0E08081816020
:10592000808381E08093EC030C943F2CE8EDF0E061
:1059300080818C7F80831092E20008951092DA00BB
:105940001092E10008951F920F920FB60F9211244A
:105950000BB60F922F933F934F935F936F937F9369
:105960008F939F93AF93BF93EF93FF938091E10049
:1059700082FF0BC08091E20082FF07C08091E100AE
:105980008B7F8093E1000E9469288091DA0080FF7C
:105990001FC08091D80080FF1BC08091DA008E7FED
:1059A0008093DA008091D90080FF0DC084E189BD29
:1059B00086E189BD09B400FEFDCF81E08093ED034F
:1059C0000E94302805C019BC1092ED030E944228A5
:1059D0008091E10080FF19C08091E20080FF15C036
:1059E0008091E2008E7F8093E2008091E2008061EE
:1059F0008093E2008091D80080628093D80019BC27
:105A000085E08093ED030E944F288091E10084FFA0
:105A100030C08091E20084FF2CC084E189BD86E122
:105A200089BD09B400FEFDCF8091D8008F7D8093A1
:105A3000D8008091E1008F7E8093E1008091E200A8
:105A40008F7E8093E2008091E20081608093E2008B
:105A50008091E903882311F084E007C08091E3007E
:105A600087FD02C081E001C083E08093ED030E94C6
:105A70005B288091E10083FF29C08091E20083FFD1
:105A800025C08091E100877F8093E10082E08093D0
:105A9000ED031092E9038091E1008E7F8093E10095
:105AA0008091E2008E7F8093E2008091E20080612D
:105AB0008093E20042E060E080E00E949E2B8091B3
:105AC000F00088608093F0000E944928FF91EF91D8
:105AD000BF91AF919F918F917F916F915F914F9106
:105AE0003F912F910F900BBE0F900FBE0F901F9004
:105AF00018951F920F920FB60F9211240BB60F92AA
:105B00002F933F934F935F936F937F938F939F93C5
:105B1000AF93BF93CF93DF93EF93FF93C091E900CF
:105B2000CF708091EC00D82FD17080FDD0E810921A
:105B3000E9008091F000877F8093F00078940E94C4
:105B4000C12D1092E9008091F00088608093F000F0
:105B5000CD2BCF70C093E900FF91EF91DF91CF91F2
:105B6000BF91AF919F918F917F916F915F914F9175
:105B70003F912F910F900BBE0F900FBE0F901F9073
:105B800018951F93CF93DF93CDB7DEB7AA970FB6C3
:105B9000F894DEBF0FBECDBFEEEEF3E08091F100D2
:105BA000819323E0E63FF207C9F70E94C328809162
:105BB000E80083FF2EC18091EE039091EF03492FFF
:105BC00050E04A30510508F024C1FA01E956FF4F70
:105BD0000C945C2F803821F0823809F01AC108C07B
:105BE0008091EA039091EB03992389F082600FC0C2
:105BF0008091F2038F70873008F00BC18093E90029
:105C00008091EB0085FB882780F91092E900909144
:105C1000E800977F9093E8008093F1001092F100E4
:105C2000D1C0282F2D7F09F0F4C0882319F08230CD
:105C300061F0EFC08091F003813009F0EAC0933049
:105C400009F080E08093EB032EC08091F003811176
:105C50002AC08091F2038F702FEF280F263008F0B2
:105C6000D8C08093E9002091EB0020FF1CC0933046
:105C700021F48091EB00806214C09091EB00906160
:105C80009093EB0021E030E0A90102C0440F551FC2
:105C90008A95E2F74093EA001092EA008091EB00C7
:105CA00088608093EB001092E9008091E800877F84
:105CB0008093E8000E94D32BACC08111AAC0109140
:105CC000F0031F778091E3008078812B8093E300BD
:105CD0008091E800877F8093E8000E94D32B809119
:105CE000E80080FFFCCF8091E30080688093E300B0
:105CF000111102C082E001C083E08093ED0389C0EE
:105D00008058823008F085C08091F0039091F103B3
:105D10008C3D53E0950779F583E08A838AE2898395
:105D20004FB7F894DE01139620E03EE051E2E32FF6
:105D3000F0E050935700E49120FF03C0E295EF702C
:105D40003F5FEF708E2F90E0EA3010F0C79601C0F1
:105D5000C0968D939D932F5F243149F74FBF80915B
:105D6000E800877F8093E8006AE270E0CE01019648
:105D70000E94E32A16C06091F2037091F303AE0112
:105D80004F5F5F4F0E942A2ABC01892B09F441C052
:105D90009091E800977F9093E80089819A810E9412
:105DA0003F2B8091E8008B778093E80032C08038E9
:105DB00081F58091E800877F8093E8008091E90376
:105DC0008093F1008091E8008E7772CF811121C01D
:105DD0008091F0039091F10399270297D4F4809178
:105DE000E800877F8093E8008091F0038093E903C7
:105DF0000E94D32B8091E903811106C08091E300BA
:105E000087FD02C081E001C084E08093ED030E9421
:105E1000AA288091E80083FF0AC08091E800877F6C
:105E20008093E8008091EB0080628093EB00AA965B
:105E30000FB6F894DEBF0FBECDBFDF91CF911F919B
:105E40000895CF938091ED038823A1F0C091E900DC
:105E5000CF709091EC00892F817090FD80E8C82B65
:105E60001092E9008091E80083FD0E94C12DCF705F
:105E7000C093E900CF910895991B79E004C0991F60
:105E8000961708F0961B881F7A95C9F78095089594
:105E900097FB072E16F4009407D077FD09D00E94D7
:105EA000652F07FC05D03EF4909581959F4F08958E
:105EB000709561957F4F0895EE0FFF1F0024001C21
:105EC0000BBE0790F691E02D0994AA1BBB1B51E174
:105ED00007C0AA1FBB1FA617B70710F0A61BB70B5A
:105EE000881F991F5A95A9F780959095BC01CD01FF
:105EF0000895FB01DC0104C08D910190801921F40B
:105F000041505040C8F7881B990B0895F999FECF6E
:105F100092BD81BDF89A992780B50895A8E1B0E0B7
:105F200042E050E00C94BA2F262FF999FECF92BD93
:105F300081BDF89A019700B4021639F01FBA20BD4E
:105F40000FB6F894FA9AF99A0FBE08950396272F80
:105F50000E94952F0E94942F252F0E94952F242F69
:105F60000C94952F0196272F0E94952F0C94942F17
:105F7000DC01CB01FC01F999FECF06C0F2BDE1BD09
:105F8000F89A319600B40D9241505040B8F70895F8
:045F9000F894FFCFB3
:105F9400C800DF02280850011E0A14019927BC27F3
:105FA4009D272C2828289C2701E200E900EA00B557
:105FB40000B600B700CD008301CC008A01920194A1
:105FC400012102230224022502260227022A02B307
:105FD40000B4006F007000818283E200E900EA00EF
:105FE400B500B600B700CD008301CC008A01920150
:105FF40094012102230224022502260227022A02F6
:10600400B300B4006F0070008182836061626364D6
:106014006566679091F09394F19697C0C1C2C3C42A
:10602400C5C630313233343536373F3F3F006D6BB0
:106034005F64656C6179006D6B5F696E746572761F
:10604400616C006D6B5F6D61785F73706565640092
:106054006D6B5F74696D655F746F5F6D6178006D02
:106064006B5F776865656C5F6D61785F737065659C
:1060740064006D6B5F776865656C5F74696D655FFF
:10608400746F5F6D61780040B622690DB30C910C9A
:06609400360C4F0C680CF5
:00000001FF
